:017F920001ED
:030033000218FBB5
:0D003600E51104907841F090C000E0FF2239
:10004600E4FF74402FF582E4347BF583E0FEE5158A
:100056002404FDE43514FAA9057B01EF7C0029F997
:10006600EC3AFAEE1211EC0FBF22D7E5152405F58E
:1000760082E43514F583E07003020134E5152409A2
:10008600F582E43514F583E0700EE515240AF58251
:10009600E43514F583E060187F01E4FD12166BE584
:1000A600152431F582E43514F583E054CFF0804110
:1000B600E5152406F582E43514F583E0FF12000306
:1000C600E5152407F582E43514F583E0FF1215AB38
:1000D6007F01E5152408F582E43514F583E0FD1269
:1000E600166BE5152431F582E43514F583E04430CA
:1000F600F0E5152439F582E43514F583E04480F003
:1000030090784174F3F090C00074BFF0907841741D
:10001300F0F090C000EFF090784174F3F0E5152410
:1000230037F582E43514F583E0547F90C000F02265
:03004300021B009D
:030000000210905B
:4001060090784174F4F0E5152439F582E43514F583E090C000F090784174F2F0E5152436F582E43514F583E0440690C000F0E515240BF582E43514F583E06032E515240C2B
:40014600F582E43514F583E0543FFFE5152437F582E43514F583EFF090784174F3F0E5152437F582E43514F583E090C000F0E515240DF582E43514F583E0700302024FE598
:40018600152417F582E43514F583E06011E5152432F582E43514F583E04404F0800FE5152432F582E43514F583E054FBF0E4FFE5152432F582E43514F583E0FD12166BE53A
:4001C60015240EF582E43514F583E06011E5152433F582E43514F583E04480F0800FE5152433F582E43514F583E0547FF0E5152433F582E43514F583E054FCF0E515240FEB
:40020600F582E43514F583E0602FE5152433F582E43514F583E04402F0E5152410F582E43514F583E0FF12160BE5152411F582E43514F583E0FF12163BE5152433F582E415
:400246003514F583E0FF1215DBE5152414F582E43514F583E06044E5152415F582E43514F583E06011E5152439F582E43514F583E04401F0800FE5152439F582E43514F55D
:4002860083E054FEF090784174F4F0E5152439F582E43514F583E090C000F0E5152412F582E43514F583E06044E5152413F582E43514F583E06011E5152439F582E43514F6
:4002C600F583E04402F0800FE5152439F582E43514F583E054FDF090784174F4F0E5152439F582E43514F583E090C000F0E5152416F582E43514F583E0FFE5152435F5821A
:40030600E43514F583EFF0E5152417F582E43514F583E030E011E5152431F582E43514F583E04440F0800FE5152431F582E43514F583E054BFF0E5152418F582E43514F576
:4003460083E0FFE515243BF582E43514F583EFF0E5152419F582E43514F583E06011E5152439F582E43514F583E04410F0800FE5152439F582E43514F583E054EFF0907869
:400386004174F4F0E5152439F582E43514F583E090C000F0E515241AF582E43514F583E0606BE5152437F582E43514F583E054BFF090784174F3F0E5152437F582E435141F
:4003C600F583E0547F90C000F090784174F1F0120036EF54FE90C000F0E5152432F582E43514F583E054FDFFF0FDE4FF12166BE515242CF582E43514F583E4F0E515242BA3
:40040600F582E43514F583E4F0E5164213E515241BF582E43514F583E0700EE5152425F582E43514F583E06028E5152432F582E43514F583E04402FFF0FDE4FF12166BE523
:4004460015242BF582E43514F5837401F0E5164213E515241CF582E43514F583E0FF700EE5152425F582E43514F583E0602A90784174F2F0E5152436F582E43514F583E0D6
:40048600440490C000F0EF600FE5152431F582E43514F583E04404F0E515241DF582E43514F583E06027E5152437F582E43514F583E04440F090784174F3F0E5152437F560
:4004C60082E43514F583E0547F90C000F0E515241EF582E43514F583E06028E5152432F582E43514F583E054FEFFF0FDE4FF12166BE515242DF582E43514F5837401F0E56B
:40050600164213E515241FF582E43514F583E0700EE5152425F582E43514F583E06027E5152432F582E43514F583E04401FFF0FDE4FF12166BE515242DF582E43514F58373
:40054600E4F0E5164213E5152420F582E43514F583E0700EE5152425F582E43514F583E0601890784174F2F0E5152436F582E43514F583E0440290C000F0E5152421F582B7
:40058600E43514F583E0600FE5152431F582E43514F583E04402F0E5152422F582E43514F583E0601FE515242EF582E43514F5837401F0E515243AF582E43514F583E4F0F0
:4005C600E5164213E5152423F582E43514F583E0600312187AE5152424F582E43514F583E06023E5152431F582E43514F583E04408F0E516C454F0FF4211907F96E04FF000
:40060600907841E04FF0E5152425F582E43514F583E06024E5152431F582E43514F583E054F7F0E516C454F0F4FF5211907F96E05FF0907841E05FF022907FE9E01211FE43
:40064600079900080D01087903066206078A08077E0907660A07750B000008C8907FEBE024FE601C1470030207142402600302075C7419907FD4F07400907FD5F00208CF4C
:40068600907FEAE004758217758319F0907FEAE030E0047F0280027F03758282758319EFF075826D758319F0758266758319F075825F758319F0758258758319F0907FEA0A
:4006C600E030E1047F6480027F3275821A758319EFF0907FEFE0FE907FEEE07C002400F518EC3EF517753319753412758214758319E0752700F528D3E5289518E5279517D6
:40070600400685172785182812130D0208CF907FEAE0FF12145FEA496032907FEEE0751700F518AE02AF018E338F348F828E83E0FEA3E08E27F528D39518E527951740068B
:4007460085172785182812130D0208CF907FB4E04401F00208CF907FB4E04401F00208CF907F00E525F0907FB57401F00208CF907FEAE0F5250208CF907FEAE0F522120A9B
:40078600CE0208CF907F00E522F0907FB57401F00208CF907FE8E0247F60241460312402705BA200E433FF25E0FFA206E4334F907F00F0E4A3F0907FB57402F00208CFE4C9
:4007C600907F00F0A3F0907FB57402F00208CF907FECE0F45480FFC4540FFFE054072F25E024B4F582E4347FF583E054FD907F00F0E4A3F0907FB57402F00208CF907FB45C
:40080600E04401F00208CF907FE8E024FE601D240260030208CF907FEAE0B40105C2000208CF907FB4E04401F00208CF907FEAE07038907FECE0F45480FFC4540FFFE05490
:40084600072F25E024B4F582E4347FF583E4F0907FECE05480FF131313541FFFE054072F907FD7F0E04420F0805F907FB4E04401F08056907FE8E024FE60182402704A90CA
:400886007FEAE0B40104D200803F907FB4E04401F08036907FEAE07020907FECE0F45480FFC4540FFFE054072F25E024B4F582E4347FF5837401F08010907FB4E04401F046
:4008C6008007907FB4E04401F0907FB4E04402F022E512540F70030209C812169AEF20E1751216F8EF14F5181218C5EF2518FFE433FEC3EF9480EE64809480505985158201
:40090600851483E0FEA3E0FFF5828E83E030E011E5152431F582E43514F583E04480F0800FE5152431F582E43514F583E0547FF0E5152431F582E43514F583E020E212E5CC
:4009460018600EF523EF2401F52DE43EF52C1214A0E4FF1214D7E5152431F582E43514F583E030E75D1218C5E515243BF582E43514F583E0FEEFC39E5048E515242FF58207
:40098600E43514F5837401F0E5152431F582E43514F583E0547BF0E515243AF582E43514F583E4F0E5164213907FC2E030E110E5152426F582E43514F583E0F524800312C5
:4009C600129C1216C9EF30E103020ACD1217C78F181218D3E5152438F582E43514F583EFF0E5152435F582E43514F583E0FFE518C39F50281218A9EF30E021E5152438F52E
:400A060082E43514F583E020E712E5152431F582E43514F583E020E103020ACDE5152431F582E43514F583E054FDF0E5187003020ACDB4800FE5152438F582E43514F583DE
:400A4600E04402F0E5152438F582E43514F583E0FF30E729E518D394204003751820851823851582851483A3A3E0FCA3E08C2CF52D1213CFE51825E0FF12150D22E518D3C3
:400A8600943F400375183F851823E5152438F582E43514F583E0FF851582851483A3A3E0FCA3E0F5828C83EFF0851582851483A3A3E0FEA3E02401F52DE43EF52C12141D4F
:400AC600E51804FF12150D22E4907F93F0907F9C74FFF0E4907F96F0907F94F090784A04F0F58E907F9574C0F0907F9E743FF0907F98742FF090784374F7F0E4907841F02C
:400B0600907FDF749FF0907FDEF0907F92E04402F07E7B7FC075147B7515C0907F98742EF0751601120F287E7B7FC075147B7515C0907F98742EF0751601E5152426F58290
:400B4600E43514F583E4F07E7E7F40851582851483747EF0A37440F07E7E7F80851582851483A3A3747EF0A37480F07E7C7F0075147C751500907F98742DF0751602120F0A
:400B8600287E7C7F0075147C751500907F98742DF0751602E5152426F582E43514F5837401F07E7D7FC0851582851483747DF0A374C0F07E7E7F00851582851483A3A374EE
:400BC6007EF0A37400F07E7C7F4075147C751540907F98742BF0751604120F287E7C7F4075147C751540907F98742BF0751604E5152426F582E43514F5837402F07E7D7F57
:400C060040851582851483747DF0A37440F07E7D7F80851582851483A3A3747DF0A37480F07E7C7F8075147C751580907F987427F0751608120F287E7C7F8075147C751590
:400C460080907F987427F0751608E5152426F582E43514F5837403F07E7C7FC0851582851483747CF0A374C0F07E7D7F00851582851483A3A3747DF0A37400F0C20AC209D3
:400C8600E4F511D20222E510045403F51014601F146031146043240370527E7B7FC075147B7515C0907F98742EF0751601803D7E7C7F0075147C751500907F98742DF07564
:400CC600160280287E7C7F4075147C751540907F98742BF075160480137E7C7F8075147C751580907F987427F0751608E53255167003020E27E516F45232E526547FFF7095
:400D060017E52A55166034907F96E0FEE516C454F0F4FDEE5DF08023BF2020E5152431F582E43514F583E030E311E4F52A907F96E0FFE516C454F0FEEF4EF0E515243AF5C3
:400D460082E43514F583E06003E014F0E5152434F582E43514F583E06003E014F0E06003020E27740AF0120036EF5401FFF518E515242CF582E43514F583E06F6007E518F1
:400D8600F0E51642131218E18F18E5152427F582E43514F583E0FFE5185410FE6F6006EEF0E5164213E5152428F582E43514F583E0FFE5185480FE6F6006EEF0E516421386
:400DC600E5152429F582E43514F583E0FFE5185420FE6F6015EEF0E5152431F582E43514F583E030E404E5164213E515242AF582E43514F583E0FFE5185440FE6F6015EE23
:400E0600F0E5152431F582E43514F583E030E504E5164213E5152430F582E43514F583E4F022300903020F27E52414602A14604114605814606F24046003020EE57E7B7F31
:400E4600C075147B7515C0907F98742EF075160112129C752401227E7C7F0075147C751500907F98742DF075160212129C752402227E7C7F4075147C751540907F98742B05
:400E8600F075160412129C752403227E7C7F8075147C751580907F987427F075160812129C75240422300433C2045313DFE4F5187E007B00742E2518F9EE3400FA1211A6CA
:400EC600FF74802518F582E4347BF583EFF00518E518B403DB907FC37403F075240522E536603BD5360A5313EF300A04D209C20AE4F5187E007B0074352518F9EE3400FACC
:400F06001211A6FF74802518F582E4347BF583EFF00518E518B403DB907FC37403F0E4F52422E4F5197E007B01E5152519F9EE3514FAE41211EC0519E519B43CE8E51524FA
:400F460035F582E43514F5837401F090784174F3F0E5152437F582E43514F5837403F090C000F07F0CE4FD12166B7F10E5152433F582E43514F583EFF01215DB9078417464
:400F8600F2F07F01E5152436F582E43514F583EFF0440690C000F090784174F4F0E5152439F582E43514F5837480F090C000F00FE4FD12166BE4FF7EA3E5152432F582E486
:400FC6003514F583EEF0FD12166B90784174F1F090C000E4F07F057D7F12166B7F011215437F037D0712166B2253133F907BF1E030E3167E7B7FC075147B7515C0907F986B
:40100600742EF07516011208D7907C31E030E3167E7C7F0075147C751500907F98742DF07516021208D7907C71E030E3167E7C7F4075147C751540907F98742BF0751604C4
:401046001208D7907CB1E030E3167E7C7F8075147C751580907F987427F07516081208D70512E512540FF517700412111C22E517B40104120C8C22907FC2E020E108E51370
:401086006004120E2822120C8C22787FE4F6D8FD7581370210D7021224E493A3F8E493A34003F68001F208DFF48029E493A3F85407240CC8C333C4540F4420C8834004F4D7
:4010C60056800146F6DFE4800B0102040810204080901845E47E019360BCA3FF543F30E509541FFEE493A360010ECF54C025E060A840B8E493A3FAE493A3F8E493A3C8C589
:4011060082C8CAC583CAF0A3C8C582C8CAC583CADFE9DEE780BE907FD2E030E1030211A5C209907B40E014602614603B14605024836064248070637E7B7FC075147B75153A
:40114600C0907F98742EF0751601120046804B7E7C7F0075147C751500907F98742DF075160212004680337E7C7F4075147C751540907F98742BF0751604120046801B7E2B
:401186007C7F8075147C751580907F987427F07516081200468003121751E4907FD3F022BB010689828A83E0225002E722BBFE02E32289828A83E49322BB010CE58229F5B8
:4011C60082E5833AF583E0225006E92582F8E622BBFE06E92582F8E222E58229F582E5833AF583E49322BB010689828A83F0225002F722BBFE01F322D083D082F8E49370B6
:4012060012740193700DA3A393F8740193F5828883E4737402936860EFA3A3A380DF907FAEE0FFD39200E433FEEF4EF0D2E843D820907FDE7401F0907FDFF0907FAB74FFC2
:40124600F0907FA9F0907FAAF05391EF907FAF7401F0907FAE740DF0D2AFD20B121809C201E4F52BF531C207C20275290F907FD8E06526600675320FE0F526300203120F8C
:40128600EF300107C20112063F80E23008DFC20812182A80D822E5135516606AE515243AF582E43514F583E0705CE516F45213E5152426FFE43514FEE4FD0FEFAA067001C7
:4012C6000E14F5828A83E0FC74802DF582E4347BF583ECF00DBD0BE2907FC3740BF0E515243AF582E43514F5837410F0E515242EF582E43514F583E4F0E515242FF582E423
:401306003514F583E4F022E52845276057AE27AF28D3EF9440EE940040047E007F40C3E5289FF528E5279EF527E4FDEDC39FE49E501F853482853383E0FC74002DF582E4BA
:40134600347FF583ECF00D0534E5347002053380DA907FA97401F0907FACE04401F0907FB5EFF022907FACE054FEF0E4907FB5F022907F98740FF0E490784AF0907F94F0E1
:40138600907F9D74FFF0E4907F97F0907841F0907F93F0907F9C74FFF0300007E529540FFF80027F00907F96EFF0907F98741FF0E4907F95F0907F9E743FF0907F9874DFAD
:4013C600F0907F92E054FDF0228F19052DE52DAE2C7002052C14F5828E83E519F01218EF052DE52DAC2C7002052C14F5828C83EFF01523E523601FE5152438F582E4351416
:40140600F583C083C082E0FE1218D38F19EE4FD082D083F080B522907841E511F090784F74C0F0E4907850F0E52C907851F0AE2CE52D907852F0907854E523F09078577470
:4014460004F0907FE2E04410F0E054F7F0E4907855F0907855E060FA228F19E4F51A751BFF751C19751D86AB1BAA1CA91D9000011211BFB4031DAF1A051AEFB519012212F9
:4014860011A67E0029FFEE3AA907751BFFF51C891D80D47B007A00790022907841E511F0E52C90784FF0AE2CE52D907850F090785174C0F0E4907852F0907854E523F0907D
:4014C60078577404F0E4907855F0907855E060FA22E5152404F582E43514F583E014600F1460131460178000907FC7EFF08013907FC9EFF0800C907FCBEFF08005907FCDED
:40150600EFF0E516422A22E5152404F582E43514F583E014600F1460131460178000907FB7EFF08013907FB9EFF0800C907FBBEFF08005907FBDEFF0E516422A22AE07E4A4
:40154600FFE5152432F582E43514F583E0547FFD12166B90784174F1F090C000EEF0E4E5152432F582E43514F583E04480FD12166B22C0E0C0F0C083C082C085C084C086A1
:40158600758600C0D075D0085391EF907FA97401F012130DD0D0D086D084D085D082D083D0F0D0E03290784174F3F090C00074BFF090784174F1F090C000EFF090784174A8
:4015C600F3F0E5152437F582E43514F583E0547F90C000F02290784174F3F090C00074BFF090784174F2F090C000EFF090784174F3F0E5152437F582E43514F583E0547FD7
:4016060090C000F02290784174F3F090C00074BFF090784174F4F090C000EFF090784174F3F0E5152437F582E43514F583E0547F90C000F02290784174F3F090C00074BF16
:40164600F090784174F6F090C000EFF090784174F3F0E5152437F582E43514F583E0547F90C000F02290784174F3F0E5152437F582E43514F583E0547F90C000F09078412F
:4016860074F7F090C000EFF090784174F5F090C000EDF022E5152404F582E43514F583E014600E1460111460148000907FC6E0FF22907FC8E0FF22907FCAE0FF22907FCC19
:4016C600E0FF22E5152404F582E43514F583E014600E1460111460148000907FB6E0FF22907FB8E0FF22907FBAE0FF22907FBCE0FF22E5152404F582E43514F583E0146000
:401706000E1460111460148000907FC7E0FF22907FC9E0FF22907FCBE0FF22907FCDE0FF22C0E0C083C082C085C084C086758600907FC4E4F05391EF907FAB7404F0D086BF
:40174600D084D085D082D083D0E032907B41E0F536431310A3E06009907FD77417F07437F0907B43E0F537A3E054F0F529E06002D20A22C0E0C083C082C085C084C08675A6
:401786008600D2015391EF907FAB7401F0D086D084D085D082D083D0E032C0E0C083C082C085C084C086758600D2085391EF907FAB7408F0D086D084D085D082D083D0E03C
:4017C600321218B7AE071218B7AD07EE6D60101218B7AE07EE6D60071218B7AD0780ECAF06227400F58690FDA57C05A3E582458370F922907FD6E04480F043870100000048
:40180600000022907FD6E04404F0E04408F0300B04E04402F07FF47E01121860907FD6E054F7F0221213771217F9907FD6E030E70A7F057E00121860121893120ACE220378
:4018460035800000032E810000C185C181C108C100C106012200012400008E178F18E5181518AE17700215174E60081217E81217E880EB22E5152404F582E43514F583E07E
:4018860004FF4410907FD7F0EF4430F022907FD6E04401F07F0D7E00121860907FD6E054FEF022E5112402907841F090C000E0FF22E5112403907841F090C000E0FF22E597
:4018C600112404907841F090C000E0FF22E5112405907841F090C000E0FF22E5112406907841F090C000E0FF22907841E511F090C000E0FF2253D8EF320012011001FFFFDE
:40190600FF40CD062A0100000102000409027400010100A032090400000EFF000000070501024000000705020240000007050302400000070504024000000705050240005B
:4019460000070506024000000705070240000007058102400001070582024000010705830240000107058402400001070585024000010705860240000107058702400001F3
:401986000403090448034B00650079007300700061006E002C002000610020006400690076006900730069006F006E0020006F006600200049006E006E006F005300790040
:4019C6007300200049006E0063002E0024034B00650079007300700061006E0020005500530041002D003400390057004C00430022035500530041002D00360035002000B5
:401A060032003000300033006A0061006E0033003100000000000000000000000000000000000000000000000000000000000000000000000000000000000000000000003E
:401A46000000000000000000000000000000000000000000000000000000000000000000000000000000000000000000000000000000000000000000000000000000000060
:401A86000000000000000000000000000000000000000000000000000000000000000000000000000000000000000000000000000000000000000000000000000000000020
:401AC6000000000000000000000000000000000000000000000000000000000000000000000000000000000000000000000000000000000000000000000002177900021B31
:151B06000400021727000217A000021B1000021B1400021578E0
:00000001FF
